:100000001200B81200CA75E0811200AB75E0201230
:10001000009E75E02012009E75E02012009E75E0A3
:100020002012009E75E02012009E75E04812009E8E
:1000300075E06912009E75E0C01200AB75E04912D0
:10004000009E75E06E12009E75E07312009E75E0D2
:100050007412009E75E07212009E75E07512009E8B
:1000600075E06312009E75E07412009E75E06112E7
:10007000009E75E06212009E75E06C12009E75E0B5
:100080006512009E75E07312009E75E02012009EBE
:1000900075E02112009E75E02012009E019CD29214
:1000A00085E0A0D290C2901200D022C29285E0A03A
:1000B000D290C2901200D022C29175E03811AB7577
:1000C000E00E11AB75E00611AB2275E00111AB2219
:0500D0007CFFDCFE22B4
:00000001FF
